:100000000C945D000C9485000C9485000C94850084
:100010000C9485000C9485000C9485000C9485004C
:100020000C9485000C9485000C9485000C9485003C
:100030000C9485000C9485000C9485000C9485002C
:100040000C946A030C9485000C9438030C941203EE
:100050000C9485000C9485000C9485000C9485000C
:100060000C9485000C9485000000000024002700FB
:100070002A0000000000250028002B0004040404CE
:100080000404040402020202020203030303030342
:10009000010204081020408001020408102001021F
:1000A00004081020000000080002010000030407FB
:1000B0000000000000000000B40311241FBECFEFB9
:1000C000D8E0DEBFCDBF11E0A0E0B1E0E6E0F1E1B5
:1000D00002C005900D92AC35B107D9F722E0ACE52E
:1000E000B1E001C01D92AC37B207E1F710E0CDE5F9
:1000F000D0E004C02197FE010E949005CC35D107C5
:10010000C9F70E94F3030C9481080C940000E1EB02
:10011000F0E02491EDE9F0E09491E9E8F0E0E49179
:10012000EE23C9F0222339F0233001F1A8F4213065
:1001300019F1223029F1F0E0EE0FFF1FEE58FF4FCA
:10014000A591B4912FB7F894EC91811126C09095A8
:100150009E239C932FBF08952730A9F02830C9F023
:10016000243049F7209180002F7D03C0209180002A
:100170002F7720938000DFCF24B52F7724BDDBCFEE
:1001800024B52F7DFBCF2091B0002F772093B000B6
:10019000D2CF2091B0002F7DF9CF9E2BDACFAF9236
:1001A000BF92CF92DF92EF92FF920F931F93CF9364
:1001B000DF936C017B018B01040F151FEB015E01C6
:1001C000AE18BF08C017D10759F06991D601ED915B
:1001D000FC910190F081E02DC6010995892B79F7FA
:1001E000C501DF91CF911F910F91FF90EF90DF90AC
:1001F000CF90BF90AF900895FC01538D448D252F73
:1002000030E0842F90E0821B930B541710F0CF96B0
:10021000089501970895FC01918D828D981761F0E2
:10022000A28DAE0FBF2FB11D5D968C91928D9F5FF9
:100230009F73928F90E008958FEF9FEF0895FC01D8
:10024000918D828D981731F0828DE80FF11D858D8B
:1002500090E008958FEF9FEF0895FC01918D228D1E
:10026000892F90E0805C9F4F821B91098F739927A3
:10027000089581E791E00E942D0121E0892B09F486
:1002800020E0822F089580E090E0892B29F00E94E1
:10029000390181110C9400000895FC01A48DA80F70
:1002A000B92FB11DA35ABF4F2C91848D90E00196B8
:1002B0008F739927848FA689B7892C93A089B189D8
:1002C0008C91837080648C93938D848D981306C079
:1002D0000288F389E02D80818F7D80830895EF92DD
:1002E000FF920F931F93CF93DF93EC0181E0888FF0
:1002F0009B8D8C8D98131AC0E889F989808185FFC0
:1003000015C09FB7F894EE89FF896083E889F98961
:1003100080818370806480839FBF81E090E0DF9163
:10032000CF911F910F91FF90EF900895F62E0B8DB6
:1003300010E00F5F1F4F0F731127E02E8C8D8E1171
:100340000CC00FB607FCFACFE889F989808185FFD8
:10035000F5CFCE010E944D01F1CFEB8DEC0FFD2FBB
:10036000F11DE35AFF4FF0829FB7F8940B8FEA8993
:10037000FB8980818062CFCFCF93DF93EC01888DA2
:100380008823B9F0AA89BB89E889F9898C9185FD10
:1003900003C0808186FD0DC00FB607FCF7CF8C919E
:1003A00085FFF2CF808185FFEDCFCE010E944D0108
:1003B000E9CFDF91CF9108958E50806480937C00C7
:1003C00080917A00806480937A0080917A0086FD23
:1003D000FCCF809178009091790008953FB7F89410
:1003E0008091610190916201A0916301B0916401DB
:1003F00026B5A89B05C02F3F19F00196A11DB11D80
:100400003FBFBA2FA92F982F8827BC01CD01620FBB
:10041000711D811D911D42E0660F771F881F991F76
:100420004A95D1F70895AF92BF92CF92DF92EF92A3
:10043000FF920F931F93CF93DF938B01D0E0C0E027
:1004400001975C018091720290917302DC01ED9141
:10045000FC910084F185E02D0995A816B906ACF051
:100460000E94EE016B017C010E94EE016C197D0976
:100470008E099F09683E734081059105A8F3219676
:100480000C171D07F9F680E001C081E0DF91CF91E4
:100490001F910F91FF90EF90DF90CF90BF90AF90A2
:1004A0000895DC01ED91FC910190F081E02D09941B
:1004B000CF93DF93EC0162E171E00E949605892BF6
:1004C00019F481E00E94870065E171E0CE010E948D
:1004D0009605892B29F480E0DF91CF910C94870059
:1004E000DF91CF9108954F925F926F927F928F929A
:1004F0009F92AF92BF92CF92DF92EF92FF920F93B3
:100500001F93CF93DF93CDB7DEB7C456D1090FB693
:10051000F894DEBF0FBECDBF85E10E94DC01582EEE
:10052000492E84E10E94DC01782E692E83E10E942D
:10053000DC01982E892E82E10E94DC01B82EA92EC2
:1005400081E10E94DC01D82EC92E80E10E94DC01ED
:10055000F82EE92E8FE00E94DC01182F092F8EE083
:100560000E94DC014F925F926F927F928F929F92D6
:10057000AF92BF92CF92DF92EF92FF920F931F93B1
:100580009F938F9389E191E09F938F938E010F5FEB
:100590001F4F1F930F930E94A9056EEF7FEF80916D
:1005A0007202909173020E9451020FB6F894DEBF5E
:1005B0000FBECDBFF12C2F2D30E0F80101900020AF
:1005C000E9F73197E01BF10B809172029091730271
:1005D0002E173F0758F4200F311FF9016081062EB6
:1005E000000C770B0E945102F394E5CF6FEF7FEF81
:1005F0000E945102CC59DF4F0FB6F894DEBF0FBEF8
:10060000CDBFDF91CF911F910F91FF90EF90DF90C1
:10061000CF90BF90AF909F908F907F906F905F90A2
:100620004F9008951F920F920FB60F9211242F939F
:100630003F934F935F936F937F938F939F93AF936A
:10064000BF93EF93FF9381E791E00E944D01FF91EB
:10065000EF91BF91AF919F918F917F916F915F913A
:100660004F913F912F910F900FBE0F901F901895B3
:100670001F920F920FB60F9211242F938F939F9377
:10068000EF93FF93E0918101F09182018081E091ED
:100690008701F091880182FD1BC0908180918A01C1
:1006A0008F5F8F7320918B01821741F0E0918A0157
:1006B000F0E0EF58FE4F958F80938A01FF91EF9104
:1006C0009F918F912F910F900FBE0F901F901895B3
:1006D0008081F4CF1F920F920FB60F9211242F93A7
:1006E0003F938F939F93AF93BF9380915D019091C0
:1006F0005E01A0915F01B091600130915C0123E047
:10070000230F2D3758F50196A11DB11D20935C01D3
:1007100080935D0190935E01A0935F01B0936001AF
:100720008091610190916201A0916301B091640197
:100730000196A11DB11D8093610190936201A09368
:100740006301B0936401BF91AF919F918F913F91ED
:100750002F910F900FBE0F901F90189526E8230F32
:100760000296A11DB11DD2CFE1E7F1E01382128202
:1007700088EE93E0A0E0B0E084839583A683B783FE
:1007800084E091E09183808385EC90E09587848775
:1007900084EC90E09787868780EC90E0918B808B4B
:1007A00081EC90E0938B828B82EC90E0958B848B34
:1007B00086EC90E0978B868B118E128E138E148EA2
:1007C000F0937302E0937202E9E6F1E089E9808335
:1007D00087E1818384E3828381E0838314821582AD
:1007E000168217820895CF93DF93CDB7DEB72C978B
:1007F0000FB6F894DEBF0FBECDBF789484B582608B
:1008000084BD84B5816084BD85B5826085BD85B5B4
:10081000816085BD80916E00816080936E00109232
:1008200081008091810082608093810080918100AD
:10083000816080938100809180008160809380003E
:100840008091B10084608093B1008091B00081609C
:100850008093B00080917A00846080937A008091C8
:100860007A00826080937A0080917A008160809320
:100870007A0080917A00806880937A001092C1009B
:10088000EDE9F0E02491E9E8F0E08491882399F023
:1008900090E0880F991FFC01E859FF4FA591B49192
:1008A000FC01EE58FF4F859194918FB7F894EC912D
:1008B000E22BEC938FBFE0918101F091820182E005
:1008C0008083E0918101F09182011082E0917D01AD
:1008D000F0917E011082E0917F01F091800180E132
:1008E000808310928901E0918501F091860186E074
:1008F0008083E0918301F091840180818061808315
:10090000E0918301F0918401808188608083E0918F
:100910008301F0918401808180688083E09183016C
:10092000F091840180818F7D808380916D0123E728
:1009300032E0309375022093740281608860809366
:100940006D0188E592E090937B0280937A026E01BC
:100950008DE0C80ED11C90E0E92E90E0F92E809138
:10096000720290917302DC01ED91FC910084F1859B
:10097000E02D0995892B09F450C080917202909165
:100980007302DC01ED91FC910284F385E02D099561
:100990008C3F09F042C064E670E085E090E00E9480
:1009A00013028823D1F18E01075F1F4F58018091F8
:1009B000720290917302DC01ED91FC910284F38547
:1009C000E02D0995F80181938F01EC15FD0579F76C
:1009D0008091720290917302DC01ED91FC9102848E
:1009E000F385E02D099589853A852B859C85809333
:1009F000650130936601209367019093680183300D
:100A000009F476C0B0F4813009F446C0E091740274
:100A1000F0917502823009F46FC0E114F10409F419
:100A20009ECF0E943901882309F499CF0E940000CB
:100A300096CF843009F462C0853079F780906601E2
:100A4000082D10E062E370E0C80102960E941302D4
:100A5000882319F38091720290917302DC01ED9169
:100A6000FC910284F385E02D09958EE0A82E82E0AA
:100A7000B82E912C8091720290917302DC01ED915D
:100A8000FC910284F385E02D8914E9F10995F501C3
:100A900081935F019394EECF88E0E9E6F1E0DE0117
:100AA000119601900D928A95E1F76EEF7FEF80919C
:100AB0007202909173020E9451028E010F5F1F4FCC
:100AC000F80161918F01062E000C770B8091720264
:100AD000909173020E945102A016B10689F76FEF40
:100AE0007FEF80917202909173020E94510295CF24
:100AF000E0917602F091770209958FCFE09178022C
:100B0000F0917902F9CF0995F801E25FFD4F10826B
:100B1000E0917A02F0917B028EE092E009957DCF20
:100B2000EE0FFF1F0590F491E02D0994FB01DC010D
:100B30008D9181341CF08B350CF4805E61916134B1
:100B40001CF06B350CF4605E861B611189F3990B08
:100B50000895AEE0B0E0EFEAF5E00C9458080D8996
:100B60001E8986E08C831A8309838FEF9FE79E831B
:100B70008D83AE01475E5F4F6F89788DCE01019600
:100B80000E94CC052F813885020F131FF8011082B7
:100B90002E96E4E00C947408ABE0B0E0E2EDF5E0F2
:100BA0000C944A087C013B018A01FC0117821682E1
:100BB000838181FFC8C1CE0101965C01F701938159
:100BC000F30193FD859193FF81913F01882309F4FF
:100BD00053C1853239F493FD859193FF81913F0193
:100BE000853229F4B70190E00E94BC07E7CF912C31
:100BF000212C312CFFE1F31538F08B3211F190F4F8
:100C0000803209F1833229F137FC3CC020ED280FF6
:100C10002A3050F536FE20C08AE0989E200D11241F
:100C2000922E06C08D3291F0803371F7689430F8BF
:100C3000F30193FD859193FF81913F018111DACFFB
:100C400021C0689431F8689432F8F2CF689433F890
:100C5000EFCF689434F8ECCFEAE02E9E200D1124FB
:100C6000222E689435F8E4CF8E3229F436FC04C184
:100C7000689436F8DDCF8C3619F4689437F8D8CFFD
:100C80008836B1F2982F9F7D95549330E0F08336EB
:100C9000A1F18337C1F1833509F063C02801F2E087
:100CA0004F0E511CF801C080D180692D70E036FCD8
:100CB00002C06FEF7FEFC6010E94A6074C01689447
:100CC00037F882010AC00C5F1F4FFFE3F9838824C5
:100CD0008394912C6501E89437F833FE2DC0522C93
:100CE0008114910471F5552009F468CFB70180E2B1
:100CF00090E00E94BC075A94F6CFF8018081898366
:100D00000E5F1F4FE4CF2801F2E04F0E511CF80197
:100D1000C080D180692D70E036FC02C06FEF7FEF9C
:100D2000C6010E94B1074C018201D5CFB70180E214
:100D300090E00E94BC072A942814190409F0B0F727
:100D4000CECFF60137FC859137FE81916F01B70157
:100D500090E00E94BC0751105A94F1E08F1A91085C
:100D6000BFCF843619F0893609F077C0F80137FE15
:100D70006BC060817181828193810C5F1F4FF32D65
:100D8000FF763F2E97FF09C09095809570956195ED
:100D90007F4F8F4F9F4F689437F82AE030E0A501CE
:100DA0000E94EC07C82ECA188C2C432C36FE0CC0AF
:100DB000E89440F8C91440F434FE05C032FC03C086
:100DC000F32DFE7E4F2E892C44FE95C0FE01EC0DC6
:100DD000F11D8081803309F087C0242D297E422EA9
:100DE000842D8870582E43FC95C040FE8FC09C2CEB
:100DF000821418F42C0C922C981844FE91C0B70160
:100E000080E390E00E94BC0742FE09C088E790E0C2
:100E100041FE02C088E590E0B7010E94BC07C914FA
:100E200008F48AC0CA94D12C9FEFC91AD90ACA0CF7
:100E3000DB1CF60182916F01B70190E00E94BC07B4
:100E4000AC14BD04B1F74FCF60817181072E000C47
:100E5000880B990B0E5F1F4F92CFD32CE894D4F8D8
:100E60002AE030E0853739F1232D297FD22E8F36C5
:100E700001F148F48835A9F0F701868197812B9616
:100E8000E2E10C946608803749F08837A9F7D4FE70
:100E900002C06894D2F820E130E00DC06894D4F824
:100EA000F6CF34FE03C0822F8660D82E20E132E0D8
:100EB00002C028E030E0F801D7FE0FC060817181E8
:100EC000828193810C5F1F4FA5010E94EC07C82E01
:100ED000CA183D2CE89437F867CF6081718190E0A3
:100EE00080E00E5F1F4FF0CF42FC02C0839478CFAA
:100EF0008394839475CF842D867809F471CFF6CFCF
:100F0000B70180E290E00E94BC0783948214C0F392
:100F1000512C73CF522C5818821408F46ECFF8CF8E
:100F2000842D867809F47BCF8BE241FE80E247FC7A
:100F30008DE2B70190E071CFB70180E390E00E94AD
:100F4000BC079A946CCF8FEF9FEF99CFFC0105906F
:100F5000615070400110D8F7809590958E0F9F1FBB
:100F60000895FC016150704001900110D8F7809500
:100F700090958E0F9F1F08950F931F93CF93DF932C
:100F8000182F092FEB018B8181FD09C01FEF0FEF97
:100F9000812F902FDF91CF911F910F91089582FFA4
:100FA00014C02E813F818C819D81281739073CF424
:100FB000E881F981CF0101969983888310838E811E
:100FC0009F8101969F838E83E3CFE885F985812FEA
:100FD0000995892BA1F3DACFFA01AA27283051F11C
:100FE000203181F1E8946F936E7F6E5F7F4F8F4F5A
:100FF0009F4FAF4FB1E03ED0B4E03CD0670F781FB9
:10100000891F9A1FA11D680F791F8A1F911DA11D9D
:101010006A0F711D811D911DA11D20D009F46894D6
:101020003F912AE0269F11243019305D3193DEF67E
:10103000CF010895462F4770405D4193B3E00FD034
:10104000C9F7F6CF462F4F70405D4A3318F0495D1F
:1010500031FD4052419302D0A9F7EACFB4E0A69502
:101060009795879577956795BA95C9F70097610524
:10107000710508959B01AC010A2E0694579547957A
:1010800037952795BA95C9F7620F731F841F951F6F
:10109000A01D08952F923F924F925F926F927F9280
:1010A0008F929F92AF92BF92CF92DF92EF92FF9278
:1010B0000F931F93CF93DF93CDB7DEB7CA1BDB0B24
:1010C0000FB6F894DEBF0FBECDBF09942A883988C9
:1010D00048885F846E847D848C849B84AA84B984D0
:1010E000C884DF80EE80FD800C811B81AA81B981DC
:1010F000CE0FD11D0FB6F894DEBF0FBECDBFED01F0
:061100000895F894FFCFF2
:10110600000000006F01CF00FC00BC012D010B01A7
:101116001F014F4E004F4646007B224130223A25A2
:10112600752C224131223A25752C224132223A254C
:10113600752C224133223A25752C224134223A2538
:10114600752C224135223A25752C224136223A2524
:0C115600752C224137223A25757D0000DF
:00000001FF
